:1000000062EF25F0FFFFFFFF0001568456AE10EFB0
:1000100000F0010E4E6E4D6A4C6A4B6A55364D32F9
:10002000FF0E1200000155AE4D9E000E12000001A1
:10003000568256AE22EF00F04E684D684C684B6811
:1000400055364D32FF0E120000014D6A4C6A4B6A64
:10005000536A4E6A000E1200000157B06FEF00F0B5
:1000600057A217EF01F0596A000E4D6486EF00F0B9
:10007000F00E4D14D8A451EF00F04D3A4C380F0B50
:100080004D264C38F00B4C6E4B380F0B4C264B3832
:10009000F00B4B6E53380F0B4B265338F00B536E4F
:1000A0005984D8904DBE6AEF00F053364B364C362B
:1000B0004D36592A4DBE6AEF00F053364B364C365A
:1000C0004D36592A4DBE6AEF00F053364B364C364A
:1000D0004D36592A59504E640BEF01F04E5E56BC16
:1000E00053AE11EF01F0D880800E53644B30000EF8
:1000F0004B224C224D22D8A011EF01F04D324C3250
:100100004B324E4A17EF01F011EF01F04CC04DF0A9
:100110004BC04CF053C04BF0536A000E59864D64EF
:10012000BDEF00F0F00E4D14D8A4A5EF00F04D3A4D
:100130004C380F0B4D264C38F00B4C6E4B380F0BD8
:100140004C264B38F00B4B6E5984D8904DBE6AEF5D
:1001500000F04B364C364D36592A4DBE6AEF00F052
:100160004B364C364D36592A4DBE6AEF00F04B36B1
:100170004C364D36592A6AEF00F04CC04DF04BC05A
:100180004CF04B6A000E599659884D64EAEF00F026
:10019000F00E4D14D8A4D5EF00F04D3A4C380F0BAB
:1001A0004D264C38F00B4C6E5984D8904DBE6AEFFA
:1001B00000F04C364D36592A4DBE6AEF00F04C36F1
:1001C0004D36592A4DBE6AEF00F04C364D36592A4D
:1001D0006AEF00F04CC04DF04C6A000E59864D6439
:1001E0001DEF01F0F00E4D14D8A4F9EF00F04D3AD8
:1001F0005984D8904DBE6AEF00F04D36592A4DBE55
:100200006AEF00F04D36592A4DBE6AEF00F04D36C8
:10021000592A6AEF00F0010E576E04EC00F021EF4E
:1002200001F0020E576E12EC00F021EF01F0040E07
:10023000576E17EC00F021EF01F0080E576E24EC1A
:1002400000F012000001586A536A4B50D8B4000CF9
:100250004F18556E55BE581E566A4FAE32EF01F01C
:100260004F1E4F2A4BA037EF01F04B1E4B2A4B502D
:100270004F10556E55BE5EEF01F04F50535E4B363A
:100280004B3453364F5053264B36060E576E4B3475
:1002900053364F504BB0535E4BA053264B36572E20
:1002A00047EF01F04BA0532656B070EF01F058AE67
:1002B000000C4B1E4B2A531E532A000C4FAE6CEF02
:1002C00001F04BBE69EF01F04B50536E4B6A57EF94
:1002D00001F04B6A4B2A000C4B1E562A3DEF01F0F1
:1002E000532A4F50535CD8A457EF01F0536A4B2A5E
:1002F0004BAE57EF01F0FF0C12000001536A546A35
:10030000000E52624E6403EF02F04D505118556ECC
:1003100052504E267E0ED8A094EF01F04E5ED8B01B
:1003200008EF02F098EF01F04E5ED8A00DEF02F05A
:100330004D8E518E4DC059F04CC056F04BC058F008
:100340004B504F02F4CF57F04C505002F4CF4BF0CB
:10035000F3CF53F04F02F3505726F4505322000EC0
:100360004B2258505002F3505726F4505322000E9F
:100370004B224D504F02F3505326F4504B224D5018
:1003800050024C6A000E4C22F3504B26F4504C2283
:1003900058505102F3505326F4504B224D6A000E30
:1003A0004C224D2256505102F3504B26F4504C2211
:1003B000000E4D2259505102F3504C26F4504D225C
:1003C0004DBEEBEF01F053364B364C364D364E06F4
:1003D000D8B40DEF02F0FEEF01F0D880800E536428
:1003E0004B30000E4B224C224D22D8A0FEEF01F0E4
:1003F0004D324C324B324E4A08EF02F055AE4D9E14
:10040000000E10EF02F0010E24EC00F010EF02F0ED
:10041000020E17EC00F010EF02F0040E04EC00F0F6
:1004200012000001536B080E576E4B3453364F5079
:10043000535ED8B01EEF02F05326D8904B36572E9D
:1004400015EF02F0120000014C34533654364F5071
:10045000535E5050D8A0503C545E4B364C360F0E75
:10046000576E4C34533654364F504BA03FEF02F08A
:10047000535E5050D8A0503C545E44EF02F05326D7
:100480005050D8B0503C54264B364C36572E31EF96
:1004900002F04BB052EF02F04F5053265050D8B0FC
:1004A000503C5426000012000001566A5686FF0E8A
:1004B00012000001568056AE66EF02F04D6A55AE4E
:1004C000FF0E4D6E4C6E4B6E55364D32FF0E1200C8
:1004D00000014D505118596E536A546A566A4E5075
:1004E00052645CEF03F05150556E518E4D8E4E505C
:1004F000566E52504E6E000E5664ACEF02F05650DF
:10050000525ED8B44DEF03F0070E52641BEF03F0B8
:10051000525E4BC053F04CC04BF04DC04CF04D6A96
:10052000524E4DEF03F05264F0EF02F0525E4BC0BA
:1005300053F04CC04BF04C6A524E4DEF03F05264F6
:10054000CEEF02F0525E4BC053F04B6A524E4DEF6D
:1005500003F05264B5EF02F055C04DF050C04CF0BE
:100560004FC04BF0536A79EF04F0030E5264C0EFB2
:1005700002F0525E53380F0B536E524E4DEF03F0A4
:10058000D8905332524E4DEF03F0D8905332524E22
:100590004DEF03F0D89053324DEF03F0030E526449
:1005A000DFEF02F0525E53380F0B536E4B38F00BF7
:1005B00053264B380F0B4B6E524E4DEF03F0D89035
:1005C0004B325332524E4DEF03F0D8904B325332F0
:1005D000524E4DEF03F0D8904B3253324DEF03F0B3
:1005E000030E526407EF03F0525E53380F0B536E45
:1005F0004B38F00B53264B380F0B4B6E4C38F00B2F
:100600004B264C380F0B4C6E524E4DEF03F0D890EA
:100610004C324B325332524E4DEF03F0D8904C32A5
:100620004B325332524E4DEF03F0D8904C324B3296
:1006300053324DEF03F0030E526438EF03F0525E75
:1006400053380F0B536E4B38F00B53264B380F0BB0
:100650004B6E4C38F00B4B264C380F0B4C6E4D3814
:10066000F00B4C264D380F0B4D6E524E4DEF03F0F4
:10067000D8904D324C324B325332524E4DEF03F044
:10068000D8904D324C324B325332524E4DEF03F034
:10069000D8904D324C324B325332546A000E59AE20
:1006A00041EF04F0531E4B1E4C1E4D1E532A4B228D
:1006B0004C224D2241EF04F05250D8A462EF03F0D7
:1006C00079EF04F0546A4DC055F04D8E518E525062
:1006D0004E5C526ED8B434EF04F0070E526402EF51
:1006E00004F0525E4F50546E50504F6E5150506E49
:1006F000516A524E34EF04F0070E5264D7EF03F004
:10070000525E4F50546E50504F6E506A524E34EFFE
:1007100004F0070E5264B5EF03F0525E4F50546E72
:100720004F6A524E34EF04F0070E52649CEF03F010
:1007300055C04DF079EF04F0030E5264A7EF03F0BB
:10074000525E54380F0B546E524E34EF04F0D89072
:100750005432524E34EF04F0D8905432524E34EFAB
:1007600004F0D890543234EF04F0030E5264C6EF14
:1007700003F0525E54380F0B546E4F38F00B542672
:100780004F380F0B4F6E524E34EF04F0D8904F326B
:100790005432524E34EF04F0D8904F325432524E0D
:1007A00034EF04F0D8904F32543234EF04F0030E9B
:1007B0005264EEEF03F0525E54380F0B546E4F3814
:1007C000F00B54264F380F0B4F6E5038F00B4F265E
:1007D00050380F0B506E524E34EF04F0D890503218
:1007E0004F325432524E34EF04F0D89050324F32E0
:1007F0005432524E34EF04F0D89050324F325432CB
:1008000034EF04F0030E52641FEF04F0525E5438CC
:100810000F0B546E4F38F00B54264F380F0B4F6EA2
:100820005038F00B4F2650380F0B506E5138F00BEC
:10083000502651380F0B516E524E34EF04F0D890C1
:10084000513250324F325432524E34EF04F0D8907D
:10085000513250324F325432524E34EF04F0D8906D
:10086000513250324F325432536A000E59AE41EF7A
:1008700004F0541E4F1E501E511E542A4F22502267
:100880005122545053264F504B2250504C2251501D
:100890004D2259BE58EF04F0D8A067EF04F04D3256
:1008A0004C324B3253324E3E67EF04F073EF04F09C
:1008B000D8B06DEF04F0000E531E4B1E4C1E4D1EA3
:1008C000532A4B224C224D22557E6DEF04F0010E2F
:1008D000576E2CEC00F07BEF04F0020E576E2CEC00
:1008E00000F07BEF04F0040E576E17EC00F07BEF86
:1008F00004F0000E576E120000001200080E566E33
:10090000FF0E556E562E01D003D0552EFED7FAD7C6
:100910001E0E556E552EFED71200100E556E552E1A
:10092000FED7000012000001556A4E50D8A4558031
:100930005250D8A455825550D8B4F7EF04F0030AAA
:10094000D8B4B0EF04F055B0ABEF04F051AEF5EF12
:1009500004F0F3EF04F04DAEF3EF04F0F5EF04F024
:100960004D50800B556E4D9E5150800B519E551829
:10097000D8B4C1EF04F05550D8B4F3EF04F0F5EF5C
:1009800004F052504E5CD8B4CBEF04F0D8A0E7EF9F
:1009900004F0EDEF04F051504D5CD8B4D5EF04F005
:1009A000D8A0E7EF04F0EDEF04F050504C5CD8B461
:1009B000DFEF04F0D8A0E7EF04F0EDEF04F04F50C4
:1009C0004B5CD8B4F7EF04F0D8B0EDEF04F055521B
:1009D000D8B4F5EF04F0F3EF04F05552D8B4F3EFC8
:1009E00004F0F5EF04F0D8801200D8901200D880FF
:1009F000D884120012003250390807E3300E325CFE
:100A000004E3010E4B6E06EF05F04B6A1200800EF8
:100A100032184B6E800E000A4B5CD8B073D1325046
:100A200000084F6E4FC032F0800E4F184B6E800E94
:100A30006E0A4B5CD8A0C0D0640E4F6E32C04BF033
:100A400022EC01F0120E4B26000E4BBEFF0E4C6E38
:100A5000000E4C22020E4F6E000E4CBEFF0E4D6E6D
:100A60004E6E4F5007E04B364B904C364D364E365F
:100A7000FF0FF8D78A0E4B264B0E4C22000E4D224C
:100A80004BC0F6FF4CC0F7FF4DC0F8FF0900F5CF93
:100A900033F00900F5CF34F00900F5CF35F0090047
:100AA000F5CF36F0640E4F6E32C04BF022EC01F001
:100AB00053C04BF00A0E4F6E22EC01F0090E4B268C
:100AC000000E4BBEFF0E4C6E000E4C22020E4F6EFF
:100AD000000E4CBEFF0E4D6E4E6E4F5007E04B3673
:100AE0004B904C364D364E36FF0FF8D78A0E4B26BC
:100AF0004B0E4C22000E4D224BC0F6FF4CC0F7FFB0
:100B00004DC0F8FF0900F5CF4BF00900F5CF4CF0D0
:100B10000900F5CF4DF00900F5CF4EF033C04FF08E
:100B200034C050F035C051F036C052F07DEC01F0C9
:100B30004BC033F04CC034F04DC035F04EC036F0F1
:100B40000A0E4F6E32C04BF022EC01F053C04BF056
:100B5000020E4F6E000E4BBEFF0E4C6E4D6E4E6E73
:100B60004F5007E04B364B904C364D364E36FF0F0C
:100B7000F8D78A0E4B264B0E4C22000E4D224BC04E
:100B8000F6FF4CC0F7FF4DC0F8FF0900F5CF4BF062
:100B90000900F5CF4CF00900F5CF4DF00900F5CF75
:100BA0004EF033C04FF034C050F035C051F036C075
:100BB00052F07DEC01F012000001800E0A0A4B6E2B
:100BC000800E32184B5C72E20A0E4F6E32C04BF050
:100BD00022EC01F0090E4B26000E4BBEFF0E4C6EB0
:100BE000000E4C22020E4F6E000E4CBEFF0E4D6EDC
:100BF0004E6E4F5007E04B364B904C364D364E36CE
:100C0000FF0FF8D78A0E4B264B0E4C22000E4D22BA
:100C10004BC0F6FF4CC0F7FF4DC0F8FF0900F5CF01
:100C200033F00900F5CF34F00900F5CF35F00900B5
:100C3000F5CF36F00A0E4F6E32C04BF022EC01F0C9
:100C400053C04BF0020E4F6E000E4BBEFF0E4C6EAB
:100C50004D6E4E6E4F5007E04B364B904C364D3636
:100C60004E36FF0FF8D78A0E4B264B0E4C22000E45
:100C70004D224BC0F6FF4CC0F7FF4DC0F8FF0900F6
:100C8000F5CF4BF00900F5CF4CF00900F5CF4DF052
:100C90000900F5CF4EF033C04FF034C050F035C0EE
:100CA00051F036C052F07DEC01F01200020E4F6E92
:100CB00032C04BF0000E32BEFF0E4C6E4D6E4E6ECB
:100CC0004F5007E04B364B904C364D364E36FF0FAB
:100CD000F8D78A0E4B264B0E4C22000E4D224BC0ED
:100CE000F6FF4CC0F7FF4DC0F8FF0900F5CF4BF001
:100CF0000900F5CF4CF00900F5CF4DF00900F5CF14
:100D00004EF012000001800E32184B6E800E6E0AFB
:100D10004B5CD8A0C0D0640E4F6E32C04BF022ECBA
:100D200001F0120E4B26000E4BBEFF0E4C6E000E55
:100D30004C22020E4F6E000E4CBEFF0E4D6E4E6EDC
:100D40004F5007E04B364B904C364D364E36FF0F2A
:100D5000F8D7BE0E4B264B0E4C22000E4D224BC038
:100D6000F6FF4CC0F7FF4DC0F8FF0900F5CF33F098
:100D70000900F5CF34F00900F5CF35F00900F5CFC3
:100D800036F0640E4F6E32C04BF022EC01F053C0CF
:100D90004BF00A0E4F6E22EC01F0090E4B26000EAE
:100DA0004BBEFF0E4C6E000E4C22020E4F6E000E1C
:100DB0004CBEFF0E4D6E4E6E4F5007E04B364B90C3
:100DC0004C364D364E36FF0FF8D7BE0E4B264B0E27
:100DD0004C22000E4D224BC0F6FF4CC0F7FF4DC019
:100DE000F8FF0900F5CF4BF00900F5CF4CF00900F2
:100DF000F5CF4DF00900F5CF4EF033C04FF034C0C1
:100E000050F035C051F036C052F07DEC01F04BC0CF
:100E100033F04CC034F04DC035F04EC036F00A0E01
:100E20004F6E32C04BF022EC01F053C04BF0020E7B
:100E30004F6E000E4BBEFF0E4C6E4D6E4E6E4F5001
:100E400007E04B364B904C364D364E36FF0FF8D7F9
:100E5000BE0E4B264B0E4C22000E4D224BC0F6FF11
:100E60004CC0F7FF4DC0F8FF0900F5CF4BF009006B
:100E7000F5CF4CF00900F5CF4DF00900F5CF4EF05D
:100E800033C04FF034C050F035C051F036C052F08E
:100E90007DEC01F01200800E0A0A4B6E800E3218B3
:100EA0004B5C72E20A0E4F6E32C04BF022EC01F046
:100EB000090E4B26000E4BBEFF0E4C6E000E4C2250
:100EC000020E4F6E000E4CBEFF0E4D6E4E6E4F501A
:100ED00007E04B364B904C364D364E36FF0FF8D769
:100EE000BE0E4B264B0E4C22000E4D224BC0F6FF81
:100EF0004CC0F7FF4DC0F8FF0900F5CF33F00900F3
:100F0000F5CF34F00900F5CF35F00900F5CF36F014
:100F10000A0E4F6E32C04BF022EC01F053C04BF082
:100F2000020E4F6E000E4BBEFF0E4C6E4D6E4E6E9F
:100F30004F5007E04B364B904C364D364E36FF0F38
:100F4000F8D7BE0E4B264B0E4C22000E4D224BC046
:100F5000F6FF4CC0F7FF4DC0F8FF0900F5CF4BF08E
:100F60000900F5CF4CF00900F5CF4DF00900F5CFA1
:100F70004EF033C04FF034C050F035C051F036C0A1
:100F800052F07DEC01F01200020E4F6E32C04BF0B9
:100F9000000E32BEFF0E4C6E4D6E4E6E4F5007E08F
:100FA0004B364B904C364D364E36FF0FF8D7BE0EB3
:100FB0004B264B0E4C22000E4D224BC0F6FF4CC070
:100FC000F7FF4DC0F8FF0900F5CF4BF00900F5CF52
:100FD0004CF00900F5CF4DF00900F5CF4EF01200AE
:100FE0006E0E325CD8A0CAD0640E4F6E32C04BF089
:100FF00011EC02F0120E4B264C6A000E4C22020E2F
:101000004F6E000E4CBEFF0E4D6E4E6E4F5007E001
:101010004B364B904C364D364E36FF0FF8D78A0E76
:101020004B264B0E4C22000E4D224BC0F6FF4CC0FF
:10103000F7FF4DC0F8FF0900F5CF4BF00900F5CFE1
:101040004CF00900F5CF4DF00900F5CF4EF0000E41
:101050004F6E000E506E000E516E7E0E526E7DEC85
:1010600001F04BC033F04CC034F04DC035F04EC0F1
:1010700036F0640E4F6E32C04BF011EC02F053C0EC
:101080004BF00A0E4F6E11EC02F0090E4B264C6A23
:10109000000E4C22020E4F6E000E4CBEFF0E4D6E27
:1010A0004E6E4F5007E04B364B904C364D364E3619
:1010B000FF0FF8D78A0E4B264B0E4C22000E4D2206
:1010C0004BC0F6FF4CC0F7FF4DC0F8FF0900F5CF4D
:1010D0004BF00900F5CF4CF00900F5CF4DF00900B9
:1010E000F5CF4EF033C04FF034C050F035C051F062
:1010F00036C052F07DEC01F04BC033F04CC034F000
:101100004DC035F04EC036F00A0E4F6E32C04BF077
:1011100011EC02F053C04BF0020E4F6E000E4C6EFD
:101120004D6E4E6E4F5007E04B364B904C364D3661
:101130004E36FF0FF8D78A0E4B264B0E4C22000E70
:101140004D224BC0F6FF4CC0F7FF4DC0F8FF090021
:10115000F5CF4BF00900F5CF4CF00900F5CF4DF07D
:101160000900F5CF4EF033C04FF034C050F035C019
:1011700051F036C052F07DEC01F012000001325007
:101180000A08D8B07FD00A0E4F6E32C04BF011EC77
:1011900002F0090E4B264C6A000E4C22020E4F6ED6
:1011A000000E4CBEFF0E4D6E4E6E4F5007E04B369C
:1011B0004B904C364D364E36FF0FF8D78A0E4B26E5
:1011C0004B0E4C22000E4D224BC0F6FF4CC0F7FFD9
:1011D0004DC0F8FF0900F5CF4BF00900F5CF4CF0FA
:1011E0000900F5CF4DF00900F5CF4EF0000E4F6E1F
:1011F000000E506E000E516E7E0E526E7DEC01F0B0
:101200004BC033F04CC034F04DC035F04EC036F01A
:101210000A0E4F6E32C04BF011EC02F053C04BF08F
:10122000020E4F6E000E4C6E4D6E4E6E4F5007E02C
:101230004B364B904C364D364E36FF0FF8D78A0E54
:101240004B264B0E4C22000E4D224BC0F6FF4CC0DD
:10125000F7FF4DC0F8FF0900F5CF4BF00900F5CFBF
:101260004CF00900F5CF4DF00900F5CF4EF033C03A
:101270004FF034C050F035C051F036C052F07DEC24
:1012800001F01200020E4F6E32C04BF0000E4C6E99
:101290004D6E4E6E4F5007E04B364B904C364D36F0
:1012A0004E36FF0FF8D78A0E4B264B0E4C22000EFF
:1012B0004D224BC0F6FF4CC0F7FF4DC0F8FF0900B0
:1012C000F5CF4BF00900F5CF4CF00900F5CF4DF00C
:1012D0000900F5CF4EF0000E4F6E000E506E000E5E
:1012E000516E7E0E526E7DEC01F0120000014B50EB
:1012F0004F02F4CF54F0F3CF53F04C505002F4CFE0
:1013000056F0F3CF55F04B505002F3505426F450A2
:101310005522E86A56224C504F02F3505426F4509E
:101320005522E86A562250AE9AEF09F04B50555CB0
:101330004C5056584CAEA1EF09F04F50555C5050F0
:10134000565853C04BF054C04CF055C04DF056C0E9
:101350004EF0120000014E505218D8A4BFEF09F011
:101360004D505118D8A4BFEF09F04C505018D8A4D4
:10137000BFEF09F04B504F18D8B4D8841200D8945E
:10138000120012000001586A546A536A4C504B1004
:10139000D8B4000C4C505018556E55BE581E566AA5
:1013A00050AED8EF09F04F1E501E4F2AD8B4502A25
:1013B0004CAEE0EF09F04B1E4C1E4B2AD8B44C2A21
:1013C0004C505010556E55BEF8EF09F023EC02F06A
:1013D00056B00FEF0AF058AE000C4B1E4C1E4B2AB5
:1013E000D8B44C2A531E541E532AD8B4542A000C85
:1013F00050AE0AEF0AF04CBE06EF0AF04C50546EA5
:101400004B50536E4C6A4B6AEBEF09F04C6A4B6AD7
:101410004B2A000C4C1E4B1E562AE6EF09F0532AAD
:10142000D8B4542A4F50535CD8A4EBEF09F0505075
:10143000545CD8A4EBEF09F0546A536A4B2AD8B431
:101440004C2A4CAEEBEF09F00000FF0C120000013B
:10145000536A546A5250D8B4BEEF0AF04E50D8B412
:10146000C3EF0AF04D505118556E4D8E518E596A8A
:101470004DC053F04CC057F04BC058F04F50585E21
:101480005050D8A0503C575E5150D8A0513C535EAC
:10149000536A576A586AD8A055EF0AF0D8904D326F
:1014A0004C324B325332010E596E52504E5ED8A020
:1014B00062EF0AF07E0E59244E26D8B0C8EF0AF02B
:1014C00068EF0AF07E0E59244E26D8A0CDEF0AF020
:1014D000180E566E5836573653364B364C364D36F8
:1014E00059364F504B5E5050D8A0503C4C5E515036
:1014F000D8A0513C4D5E5134591259A083EF0AF0E7
:1015000058808EEF0AF04F504B265050D8B0503CC8
:101510004C265150D8B051284D265890562E6AEF7F
:101520000AF0B4EF0AF0D8904B364C364D365936A7
:101530004F504B5E5050D8A0503C4C5E5150D8A0FC
:10154000513C4D5E51345910010B5826D8B0572AE2
:10155000D8B4532AD8A4B4EF0AF0533257325832D1
:101560004E2AD8B4C8EF0AF055AE539E53504D6E74
:1015700057504C6E58504B6ED0EF0AF0010E54ECA1
:1015800002F0D0EF0AF0020E24EC00F0D0EF0AF0E7
:10159000040E17EC00F0D0EF0AF0080E04EC00F097
:1015A00012000001566A576A556A536A4E50D8B401
:1015B0005AEF0BF04D8E9E0E4E5E4EBEE5EF0AF0DA
:1015C000D8B4E5EF0AF04AEF0BF04E6C080E4E5C13
:1015D000D8A017EF0BF04E6E53364BC053F04CC0F3
:1015E0004BF04DC04CF04D6A080E4E5CD8A017EF82
:1015F0000BF04E6E53364BC053F04CC04BF04C6A60
:10160000080E4E5CD8A017EF0BF04E6E53364BC051
:1016100053F04B6A080E4E5CD8A017EF0BF04E6EDD
:101620005336536A4E50D8A4D89023EF0BF04E5047
:10163000D8B423EF0BF0D8904D324C324B325332AA
:101640004E2E1BEF0BF056BC53A034EF0BF0D8A07E
:1016500034EF0BF0532AD8B44B2AD8B44C2AD8B460
:101660004D2A4DBE5EEF0BF055AE5AEF0BF04D1EFE
:101670004C1E4B1E531E532AD8B44B2AD8B44C2AA6
:10168000D8B44D2A5AEF0BF04D6A4C6A4B6A536A34
:101690005AEF0BF0568056AE64EF0BF04D6A55AE24
:1016A00064EF0BF04D6E4C6E4B6E536E55364D32F3
:1016B00064EF0BF0000E576A65EF0BF0010E576EEA
:1016C00059EC02F065EF0BF0FF0E4D504E6E4C5092
:1016D0004D6E4B504C6E53504B6E120000014B50F0
:1016E000536E4C504B6E4D504C6E4E504D6E4E6A7C
:1016F000566A576A9E0E4E6E556A020E576E2CEC55
:1017000000F012000001517E68EC02F012000001AE
:10171000566A556A546A536A596A4E3453364F5062
:10172000535E5050D8A0503C545E5150D8A0513C0C
:10173000555E5250D8A0523C565EE86AD8A0010EC1
:10174000595E4E36070E576E4E3453365436553664
:10175000563659364F504EA0C1EF0BF0535E5050E5
:10176000D8A0503C545E5150D8A0513C555E5250C8
:10177000D8A0523C565EE86AD8A0010E595ED2EF5E
:101780000BF053265050D8B0503C54265150D8B08E
:10179000513C55265250D8B0523C5626E86AD8B033
:1017A000010E59264E36572EA4EF0BF04D3453360A
:1017B00054365536563659364F504EA0F3EF0BF08F
:1017C000535E5050D8A0503C545E5150D8A0513C6C
:1017D000555E5250D8A0523C565EE86AD8A0010E21
:1017E000595E04EF0CF053265050D8B0503C5426AC
:1017F0005150D8B0513C55265250D8B0523C562684
:10180000E86AD8B0010E59264D36070E576E4D3492
:10181000533654365536563659364F504DA024EF70
:101820000CF0535E5050D8A0503C545E5150D8A09C
:10183000513C555E5250D8A0523C565EE86AD8A042
:10184000010E595E35EF0CF053265050D8B0503C85
:1018500054265150D8B0513C55265250D8B0523C25
:101860005626E86AD8B0010E59264D36572E07EF96
:101870000CF04C34533654365536563659364F5094
:101880004DA056EF0CF0535E5050D8A0503C545E23
:101890005150D8A0513C555E5250D8A0523C565E93
:1018A000E86AD8A0010E595E67EF0CF0532650503D
:1018B000D8B0503C54265150D8B0513C55265250C7
:1018C000D8B0523C5626E86AD8B0010E59264C369C
:1018D000070E576E4C3453365436553656365936F5
:1018E0004F504CA087EF0CF0535E5050D8A0503CA6
:1018F000545E5150D8A0513C555E5250D8A0523C35
:10190000565EE86AD8A0010E595E98EF0CF0532697
:101910005050D8B0503C54265150D8B0513C552668
:101920005250D8B0523C5626E86AD8B0010E59261B
:101930004C36572E6AEF0CF04B345336543655362E
:10194000563659364F504CA0B9EF0CF0535E5050FC
:10195000D8A0503C545E5150D8A0513C555E5250D6
:10196000D8A0523C565EE86AD8A0010E595ECAEF74
:101970000CF053265050D8B0503C54265150D8B09B
:10198000513C55265250D8B0523C5626E86AD8B041
:10199000010E59264B36070E576E4B3453365436CC
:1019A0005536563659364F504BA0EAEF0CF0535E81
:1019B0005050D8A0503C545E5150D8A0513C555E78
:1019C0005250D8A0523C565EE86AD8A0010E595E2B
:1019D000FBEF0CF053265050D8B0503C54265150D9
:1019E000D8B0513C55265250D8B0523C5626E86AE1
:1019F000D8B0010E59264B36572ECDEF0CF04BB018
:101A000010EF0DF04F5053265050D8B0503C542694
:101A10005150D8B0513C55265250D8B0523C562661
:101A200012000001566A576A536A4E50D8B496EFB6
:101A30000DF04DC055F04D8E9E0E4E5E4EAE86EFB3
:101A40000DF04E6C080E4E5CD8A053EF0DF04E6EAC
:101A500053364BC053F04CC04BF04DC04CF04D6A68
:101A6000080E4E5CD8A053EF0DF04E6E53364BC0AF
:101A700053F04CC04BF04C6A080E4E5CD8A053EFAC
:101A80000DF04E6E53364BC053F04B6A080E4E5C51
:101A9000D8A053EF0DF04E6E5336536A4E50D8A473
:101AA000D8905FEF0DF04E50D8B45FEF0DF0D890A6
:101AB0004D324C324B3253324E2E57EF0DF056BC56
:101AC00053A070EF0DF0D8A070EF0DF0532AD8B4EA
:101AD0004B2AD8B44C2AD8B44D2A4DBE9AEF0DF0FB
:101AE00055AE96EF0DF04D1E4C1E4B1E531E532A45
:101AF000D8B44B2AD8B44C2AD8B44D2A96EF0DF05E
:101B00004D6A4C6A4B6A536A96EF0DF0568056AE9A
:101B1000A1EF0DF04D6A55AEA1EF0DF04D6E4C6E7C
:101B20004B6E536E55364D32A1EF0DF0576A000ED5
:101B3000A2EF0DF0010E576E000E59EC02F0A2EF6D
:101B40000DF0FF0E4D504E6E4C504D6E4B504C6E86
:101B500053504B6E12000150021000E001C0E9FF2B
:101B600002C0EAFF325200E0EF96EF9EEF9CEF9A40
:101B7000EF98EF9432BEEF8E32BCEF8C32BAEF8A20
:101B800032B8EF880050010A03E1EF94C9EF0DF07D
:101B9000EF84EF867CEC04F0325200E0EF96EF9E8B
:101BA000EF9CEF9AEF98EF9432B6EF8E32B4EF8C51
:101BB00032B2EF8A32B0EF880050010A03E1EF94AD
:101BC000E3EF0DF0EF84EF867CEC04F0EF9600502D
:101BD000010A03E17EEC04F002D08DEC04F0120067
:101BE0000001576A596A4D50D8A40AEF0EF04CC054
:101BF0004DF04BC04CF04B6A59864D50D8A40AEFBB
:101C00000EF04CC04DF04C6A599659884D50D8B4DE
:101C10001CEF0EF059504E5ED8A4D8A022EF0EF063
:101C2000D8904DBE28EF0EF04B364C364D364E2E2A
:101C300011EF0EF022EF0EF0010E576E24EC00F0C3
:101C40002CEF0EF0020E576E04EC00F02CEF0EF0AD
:101C5000040E576E12EC00F012002A0E306E000EC9
:101C6000316E030E3024E96E000E3120EA6EEECFA5
:101C70004BF07E0E4B5E4C6A000E4C5A2EC0E1FFBC
:101C80002FC0E2FF4BC0E6FF4CC0E6FF030E30243E
:101C9000E16E000E3120E26E7E0EE66E2AC04BF041
:101CA0002BC04CF02CC04DF02DC04EF012002A0E6F
:101CB000306E000E316E030E3024E96E000E3120BE
:101CC000EA6EEECF4BF04B502E244F6E000E2F20BD
:101CD000506E4FC02EF050C02FF0800E50184B6E3B
:101CE000800E4B5C02E1000E4F5C05E24B6A4C6AD1
:101CF0004D6A4E6A1200800E4B6E800E2F184B5CA0
:101D000002E12E50FF0826E24F6A506A516A526A79
:101D10002AC04BF02BC04CF02CC04DF02DC04EF023
:101D200093EC04F0010ED8B0000E4B6E4B5209E05C
:101D3000FF0E4B6EFF0E4C6EFF0E4D6EFF0E4E6E85
:101D40001200FF0E4B6EFF0E4C6E7F0E4D6EFF0E9F
:101D50004E6E12000001030E3024E16E000E3120A1
:101D6000E26E2EC0E6FF2AC04BF02BC04CF02CC018
:101D70004DF02DC04EF01200280E0101196F6E0EAD
:101D80001A6F750E1B6F6C0E1C6F6C0E1D6F290E7B
:101D90001E6F1F6B276B286B256B266B2CC04BF0BF
:101DA0002DC04CF02EC04DF0010E2C26000E2D2221
:101DB0002E224BC0F6FF4CC0F7FF4DC0F8FF0900C4
:101DC000F5CF4BF04BC022F14B52D8B4E4EF1FF0EB
:101DD00001012251250A0BE02AC0E1FF2BC0E2FFDE
:101DE00022C1E6FF2A4A2B2A274B282BD7D70101ED
:101DF000236B246B256B266B28D001012587010EF0
:101E00002C26000E2D222E225ED001012581010EEE
:101E10002C26000E2D222E2256D001012583010EE4
:101E20002C26000E2D222E224ED001012687010ED7
:101E30002C26000E2D222E2246D001012585010ED2
:101E40002C26000E2D222E223ED02CC0F6FF2DC0B7
:101E5000F7FF2EC0F8FF0900F5CF33F10101335130
:101E60002D0ACBE02CC0F6FF2DC0F7FF2EC0F8FFE7
:101E70000900F5CF33F13351200AC7E02CC0F6FF3B
:101E80002DC0F7FF2EC0F8FF0900F5CF33F1335115
:101E90002B0AC3E02CC0F6FF2DC0F7FF2EC0F8FFC1
:101EA0000900F5CF33F13351230ABFE02CC0F6FF10
:101EB0002DC0F7FF2EC0F8FF0900F5CF33F13351E5
:101EC000300ABBE001D098D7010125B3259101016B
:101ED00025B725952CC0F6FF2DC0F7FF2EC0F8FFC3
:101EE0000900F5CF4BF0000E4C6E4BC032F0FBEC0E
:101EF00004F04B5238E00101236B246B23C14BF0FB
:101F000024C14CF00A0E4F6E000E506E76EC09F0B4
:101F10002CC0F6FF2DC0F7FF2EC0F8FF0900F5CF4B
:101F200033F1010133514B24236F000E4C20246FF9
:101F3000300E235F000E245B010E2C26000E2D2296
:101F40002E222CC0F6FF2DC0F7FF2EC0F8FF09008F
:101F5000F5CF4BF0000E4C6E4BC032F0FBEC04F0B2
:101F60004B52CCE136D02CC0F6FF2DC0F7FF2EC06F
:101F7000F8FF0900F5CF33F1010133512A0A29E1B5
:101F80002FC0E9FF30C0EAFFEECF4BF0EECF4CF0B0
:101F90004BC0E9FF4CC0EAFFEECF23F1EECF24F1B6
:101FA0002FC0E9FF30C0EAFFEECF4BF0EECF4CF090
:101FB000020E4B26000E4C222FC0E1FF30C0E2FF84
:101FC0004BC0E6FF4CC0E6FF010E2C26000E2D2272
:101FD0002E222CC0F6FF2DC0F7FF2EC0F8FF0900FF
:101FE000F5CF33F1010133512E0A75E1010E2C2694
:101FF000000E2D222E222CC0F6FF2DC0F7FF2EC082
:10200000F8FF0900F5CF33F133512A0A2AE12FC036
:10201000E9FF30C0EAFFEECF4BF0EECF4CF04BC003
:10202000E9FF4CC0EAFFEECF20F1EECF21F12FC047
:10203000E9FF30C0EAFFEECF4BF0EECF4CF0020EDE
:102040004B26000E4C222FC0E1FF30C0E2FF4BC0F8
:10205000E6FF4CC0E6FF010E2C26000E2D222E229C
:1020600038D00101206B216B2CC0F6FF2DC0F7FF8B
:102070002EC0F8FF0900F5CF4BF0000E4C6E4BC0A0
:1020800032F0FBEC04F04B5224E020C14BF021C1B4
:102090004CF00A0E4F6E000E506E76EC09F02CC01C
:1020A000F6FF2DC0F7FF2EC0F8FF0900F5CF33F182
:1020B000010133514B24206F000E4C20216F300E54
:1020C000205F000E215B010E2C26000E2D222E22F9
:1020D000CBD7010104D00101206B216B26892CC0D4
:1020E0004BF02DC04CF02EC04DF0010E2C26000EF2
:1020F0002D222E224BC0F6FF4CC0F7FF4DC0F8FF3B
:102100000900F5CF22F101D127C14BF028C14CF0D5
:10211000120001012589E3D70101268532D1010191
:10212000258B010126812DD1010126832AD10101B0
:10213000258D27D126D10101258B0101258F21D1A4
:102140002FC0E9FF30C0EAFFEECF4BF0EECF4CF0EE
:102150004BC0E9FF4CC0EAFFEECF2FF1EECF30F1DC
:102160002FC0E9FF30C0EAFFEECF4BF0EECF4CF0CE
:10217000020E4B26000E4C222FC0E1FF30C0E2FFC2
:102180004BC0E6FF4CC0E6FF000E0101301902E132
:10219000000E2F1905E1190E01012F6F010E306F8E
:1021A0000101316B326B010131512F25E96E325142
:1021B0003021EA6EEECF4BF04B5203E0314B322B25
:1021C000F2D70101205121110AE03251215D02E1D3
:1021D0003151205D04E220C131F121C132F1010110
:1021E0002451325D02E12351315D06E2010131519A
:1021F000235F3251245B03D00101236B246B010167
:1022000025B717D023C14BF024C14CF0010E0101BA
:10221000235F000E245B4B504C100BE02AC0E1FF03
:102220002BC0E2FF200EE66E2A4A2B2A274B282BD2
:10223000E9D731C14BF032C14CF0010E0101315FE1
:10224000000E325B4B504C1013E02FC1E9FF30C140
:10225000EAFFEECF4BF02AC0E1FF2BC0E2FF4BC0FC
:10226000E6FF2A4A2B2A2F4B302B274B282BE1D76E
:10227000010125A717D023C14BF024C14CF0010E5A
:102280000101235F000E245B4B504C100BE02AC071
:10229000E1FF2BC0E2FF200EE66E2A4A2B2A274BD5
:1022A000282BE9D77BD52FC0E9FF30C0EAFFEECF5E
:1022B0004BF0EECF4CF04BC0E9FF4CC0EAFFEECF45
:1022C00022F12FC0E9FF30C0EAFFEECF4BF0EECF96
:1022D0004CF0020E4B26000E4C222FC0E1FF30C006
:1022E000E2FF4BC0E6FF4CC0E6FF220E01012F6F5C
:1022F000010E306F010E316F000E326F62D7C00ECB
:1023000001012513000E26133CD001012251000AC1
:10231000D8B4FAD622516C0AD8B4FBD62251660A38
:10232000D8B4FAD62251450AD8B4F9D62251650A52
:10233000D8B4F7D62251670AD8B4F6D622516F0A1C
:10234000D8B4F5D62251640AD8B4F4D62251690A19
:10235000D8B4F0D62251700AD8B4EDD62251580A1A
:10236000D8B4E9D62251780AD8B4E7D62251730AF4
:10237000D8B4E6D62251630A96E02251750ABFE02E
:10238000B4D7000E010125154B6E2651070B4C6E7C
:102390004B504C10D8B43BEF1BF026A904D0060ECE
:1023A000206F000E216F2FC0E9FF30C0EAFFEECF93
:1023B0004BF0EECF4CF04BC0E9FF4CC0EAFFEECF44
:1023C00029F1EECF2AF1EECF2BF1EECF2CF12FC079
:1023D000E9FF30C0EAFFEECF4BF0EECF4CF0040E39
:1023E0004B26000E4C222FC0E1FF30C0E2FF4BC055
:1023F000E6FF4CC0E6FF4F6A506A516A526A29C133
:102400004BF02AC14CF02BC14DF02CC14EF093EC97
:1024100004F0010ED8B0000E4B6E4B5206E00101E5
:102420002B7F030E2513000E261301012D6B2E6B3F
:1024300029C14BF02AC14CF02BC14DF02CC14EF0FC
:102440004F6A506A516A526AAAEC09F0000ED8A489
:10245000010E4B6E4B52D8B499D02CC14BF04C6A44
:102460004D6A4E6AFF0E4B140101376F000E386F34
:10247000000E38177E0E336F000E346F356F366FD7
:102480003351375D4B6E345138594C6E4BC02DF182
:102490004CC02EF1010E4B5C2D6F000E4C582E6F70
:1024A0002DC14BF02EC14CF0030E4F6E000E506E3E
:1024B00076EC09F04BC02DF14CC02EF10A0E4F6E98
:1024C000000E506EC2EC09F04BC02DF14CC02EF145
:1024D000800E4C180101336F800E335D02E1000E57
:1024E0004B5C04E2010E2D5F000E2E5B2D510008A7
:1024F000326E07EC05F029C14FF02AC150F02BC114
:1025000051F02CC152F07DEC01F04BC02FF14CC0CA
:1025100030F14DC031F14EC032F1000E4F6E000E61
:10252000506E000E516E7F0E526E2FC14BF030C1B7
:102530004CF031C14DF032C14EF093EC04F0010E7D
:10254000D8B0000E4B6E4B5206E0010E01012D5F1C
:10255000000E2E5B1BD0000E4F6E000E506E200E34
:10256000516E820E526E2FC14BF030C14CF031C112
:102570004DF032C14EF093EC04F0000ED8B0010ED5
:102580004B6E4B5203E001012D4B2E2B0101800EAF
:102590004B6E800E01012E194B5C02E12D5100089B
:1025A00004E3010E0101226F02D02DC122F10101CD
:1025B00026B119D026A315D0800E2E194B6E7F0E92
:1025C0004B5C02E1FC0E2D5D0BE3800E01012E1928
:1025D0004B6E800E21194B5C02E120512D5D01E311
:1025E00002D031EF17F001012051211107E026A39D
:1025F00005D0010E0101205F000E215B000E4B6E25
:10260000010121514B5C02E12051080804E2080E4F
:102610000101226F02D020C122F129C14BF02AC151
:102620004CF02BC14DF02CC14EF04F6A506A516AEC
:10263000526AAAEC09F0000ED8A4010E4B6E4B5260
:10264000D8B460D12DC132F007EC05F04BC04FF08B
:102650004CC050F04DC051F04EC052F029C14BF06B
:102660002AC14CF02BC14DF02CC14EF027EC0AF0E2
:102670004BC029F14CC02AF14DC02BF14EC02CF1BA
:10268000010122510008326E07EC05F04BC04FF0FB
:102690004CC050F04DC051F04EC052F029C14BF02B
:1026A0002AC14CF02BC14DF02CC14EF027EC0AF0A2
:1026B0004BC033F14CC034F14DC035F14EC036F152
:1026C00033C129F134C12AF135C12BF136C12CF1C6
:1026D00033C14BF034C14CF035C14DF036C14EF032
:1026E000D1EC0AF06EEC0BF04BC04FF04CC050F048
:1026F0004DC051F04EC052F033C14BF034C14CF0DC
:1027000035C14DF036C14EF082EC0BF0000E4F6E2D
:10271000000E506E000E516E7E0E526E93EC04F061
:10272000000ED8B0010E4B6E4B521AE029C14BF08F
:102730002AC14CF02BC14DF02CC14EF0000E4F6E53
:10274000000E506E000E516E7E0E526E68EC02F05E
:102750004BC029F14CC02AF14DC02BF14EC02CF1D9
:1027600029C14BF02AC14CF02BC14DF02CC14EF0C9
:10277000D1EC0AF04BC037F14CC038F14DC039F103
:102780004EC03AF101012251010F4B6E4C6A000E0E
:102790004C22020E4F6E000E4CBEFF0E4D6E4E6E62
:1027A0004F5007E04B364B904C364D364E36FF0FB0
:1027B000F8D7F20E4B264B0E4C22000E4D224BC08A
:1027C000F6FF4CC0F7FF4DC0F8FF0900F5CF33F11D
:1027D0000900F5CF34F10900F5CF35F10900F5CF47
:1027E00036F136513A5D08E13551395D05E1345134
:1027F000385D02E13351375D1EE329C14BF02AC138
:102800004CF02BC14DF02CC14EF0CD0E4F6ECC0EC6
:10281000506E4C0E516E7B0E526E7DEC01F04BC033
:1028200029F14CC02AF14DC02BF14EC02CF1010111
:102830002D4B2E2B67D029C14BF02AC14CF02BC158
:102840004DF02CC14EF0D1EC0AF04BC037F14CC02A
:1028500038F14DC039F14EC03AF1020E4F6E22C12F
:102860004BF0000E4C6E4D6E4E6E4F5007E04B36E7
:102870004B904C364D364E36FF0FF8D7F20E4B26A6
:102880004B0E4C22000E4D224BC0F6FF4CC0F7FF02
:102890004DC0F8FF0900F5CF33F10900F5CF34F151
:1028A0000900F5CF35F10900F5CF36F101013651B8
:1028B0003A5D08E13551395D05E13451385D02E199
:1028C0003351375D1FE229C14BF02AC14CF02BC1B7
:1028D0004DF02CC14EF0000E4F6E000E506E200ECB
:1028E000516E820E526E7DEC01F04BC029F14CC04E
:1028F0002AF14DC02BF14EC02CF1010E01012D5FCC
:10290000000E2E5B010126A39AD026B798D0800E28
:10291000000A4B6E800E010121194B5C02E120512F
:102920000A0805E20A0E0101206F000E216F29C17D
:102930004BF02AC14CF02BC14DF02CC14EF0D1EC24
:102940000AF04BC02FF14CC030F14DC031F14EC0F8
:1029500032F101012F5130113111321144E00A0ED0
:102960004F6E000E506E516E526E2FC14BF030C143
:102970004CF031C14DF032C14EF087EC0BF053C03A
:102980004BF054C04CF055C04DF056C04EF0000E08
:102990000101336F4E1808E133514D1805E13351F1
:1029A0004C1802E14B50000A1EE1010E0101205FAC
:1029B000000E215B0A0E4F6E000E506E516E526E6D
:1029C0002FC14BF030C14CF031C14DF032C14EF04F
:1029D00087EC0BF04BC02FF14CC030F14DC031F102
:1029E0004EC032F1B6D7800E010121194B6E800E18
:1029F0004B5C02E12251205D22E201012051225D67
:102A0000326E07EC05F04BC04FF04CC050F04DC09B
:102A100051F04EC052F029C14BF02AC14CF02BC1ED
:102A20004DF02CC14EF027EC0AF04BC029F14CC000
:102A30002AF14DC02BF14EC02CF120C122F1000132
:102A4000050E010120254B6E000E21214C6E4B50CE
:102A5000235F4C50245B2051211102E126A704D0B2
:102A6000010E235F000E245B030E25154B6E26C15D
:102A70004CF0000E4C164B504C1004E0010E235F3E
:102A8000000E245B25A549D025A31AD0010E2515DB
:102A90004B6E26C14CF0000E4C164B504C1003E010
:102AA0002D0E4B6E02D02B0E4B6E2AC0E1FF2BC0B9
:102AB000E2FF4BC0E6FF2A4A2B2A274B282B14D0D3
:102AC000010E25154B6E26C14CF0000E4C164B50D6
:102AD0004C100AE02AC0E1FF2BC0E2FF200EE66E98
:102AE0002A4A2B2A274B282B800E4B6E800E241946
:102AF0004B5C02E1235100080FE22AC0E1FF2BC02A
:102B0000E2FF300EE66E2A4A2B2A274B282B010EB5
:102B1000235F000E245BE8D74AD025B718D0800E7B
:102B20004B6E800E24194B5C02E1235100080FE22A
:102B30002AC0E1FF2BC0E2FF200EE66E2A4A2B2AB4
:102B4000274B282B010E235F000E245BE8D725A31B
:102B50001AD0010E25154B6E26C14CF0000E4C16F6
:102B60004B504C1003E02D0E4B6E02D02B0E4B6ED3
:102B70002AC0E1FF2BC0E2FF4BC0E6FF2A4A2B2A06
:102B8000274B282B14D0010E25154B6E26C14CF077
:102B9000000E4C164B504C100AE02AC0E1FF2BC02F
:102BA000E2FF200EE66E2A4A2B2A274B282B29C14A
:102BB0004BF02AC14CF02BC14DF02CC14EF0D1ECA2
:102BC0000AF04BC02FF14CC030F14DC031F14EC076
:102BD00032F1020E4F6E22C14BF0000E4C6E4D6E64
:102BE0004E6E4F5007E04B364B904C364D364E36BE
:102BF000FF0FF8D7F20E4B264B0E4C22000E4D2243
:102C00004BC0F6FF4CC0F7FF4DC0F8FF0900F5CFF1
:102C10004FF00900F5CF50F00900F5CF51F0090051
:102C2000F5CF52F02FC14BF030C14CF031C14DF017
:102C300032C14EF087EC0BF0300E4B262AC0E1FF7C
:102C40002BC0E2FF4BC0E6FF2A4A2B2A0101274B8B
:102C5000282B2051211102E126A776D02AC0E1FFBE
:102C60002BC0E2FF2E0EE66E2A4A2B2A0101274BCB
:102C7000282B2251205F000E215B0101225352E0DC
:102C80002207020E4F6E22C14BF0000E4C6E4D6EAD
:102C90004E6E4F5007E04B364B904C364D364E360D
:102CA000FF0FF8D7F20E4B264B0E4C22000E4D2292
:102CB0004BC0F6FF4CC0F7FF4DC0F8FF0900F5CF41
:102CC0004FF00900F5CF50F00900F5CF51F00900A1
:102CD000F5CF52F02FC14BF030C14CF031C14DF067
:102CE00032C14EF087EC0BF00A0E4F6E000E506EA4
:102CF000516E526E87EC0BF053C04BF054C04CF049
:102D000055C04DF056C04EF0300E4B262AC0E1FFA4
:102D10002BC0E2FF4BC0E6FF2A4A2B2A0101274BBA
:102D2000282BABD7205121110FE02AC0E1FF2BC087
:102D3000E2FF300EE66E2A4A2B2A274B282B010E83
:102D4000205F000E215BEED725AB0BD02AC0E1FF40
:102D50002BC0E2FF450EE66E2A4A2B2A274B282B72
:102D60000AD02AC0E1FF2BC0E2FF650EE66E2A4AB8
:102D70002B2A274B282B800E2E194B6E800E4B5C76
:102D800002E1000E2D5D12E22D5100082D6F2EC1C3
:102D90002EF1E86A2E572AC0E1FF2BC0E2FF2D0E6C
:102DA000E66E2A4A2B2A274B282B0AD02AC0E1FF9D
:102DB0002BC0E2FF2B0EE66E2A4A2B2A274B282B2C
:102DC0000A0E4F6E000E506E2DC14BF02EC14CF00E
:102DD000C2EC09F0300E4B262AC0E1FF2BC0E2FF07
:102DE0004BC0E6FF2A4A2B2A0101274B282B0A0E4B
:102DF0004F6E000E506E2DC14BF02EC14CF0C2EC48
:102E000009F053C04BF054C04CF0300E4B262AC092
:102E1000E1FF2BC0E2FF4BC0E6FF2A4A2B2A01014B
:102E2000274B282B25A71BD0800E4B6E800E241914
:102E30004B5C02E12351000812E22AC0E1FF2BC0E3
:102E4000E2FF200EE66E2A4A2B2A0101274B282B8F
:102E5000010E235F000E245B23512411EEE1CEEF1F
:102E60000EF0010126A3FFD0800E2E194B6E800EAE
:102E70004B5C02E1000E2D5D0BE2010E01012D5DA8
:102E80004B6E000E2E594C6E4B50205F4C50215B08
:102E900029C14BF02AC14CF02BC14DF02CC14EF092
:102EA000D1EC0AF04BC02FF14CC030F14DC031F1E4
:102EB0004EC032F1010E0101226F010122510A0AB6
:102EC00039E0020E4F6E22C14BF0000E4C6E4D6E7B
:102ED0004E6E4F5007E04B364B904C364D364E36CB
:102EE000FF0FF8D7F20E4B264B0E4C22000E4D2250
:102EF0004BC0F6FF4CC0F7FF4DC0F8FF0900F5CFFF
:102F000033F10900F5CF34F10900F5CF35F10900AF
:102F1000F5CF36F101013651325D08E13551315DB1
:102F200005E13451305D02E133512F5D03E30101CE
:102F3000222BC3D701012251205D376F000E21598A
:102F4000386F37C120F138C121F12FC14BF030C1AA
:102F50004CF031C14DF032C14EF06EEC0BF04BC075
:102F60004FF04CC050F04DC051F04EC052F029C14E
:102F70004BF02AC14CF02BC14DF02CC14EF082EC2D
:102F80000BF04BC033F14CC034F14DC035F14EC0A5
:102F900036F137C132F007EC05F033C14FF034C1E0
:102FA00050F035C151F036C152F07DEC01F0000E09
:102FB0004F6E000E506E000E516E7E0E526E68EC1B
:102FC00002F0D1EC0AF04BC02FF14CC030F14DC0F3
:102FD00031F14EC032F101012051211144E00A0EBD
:102FE0004F6E000E506E516E526E2FC14BF030C1BD
:102FF0004CF031C14DF032C14EF087EC0BF053C0B4
:103000004BF054C04CF055C04DF056C04EF0000E81
:103010000101336F4E1808E133514D1805E133516A
:103020004C1802E14B50000A1EE10A0E4F6E000ED2
:10303000506E516E526E2FC14BF030C14CF031C109
:103040004DF032C14EF087EC0BF04BC02FF14CC06D
:1030500030F14DC031F14EC032F1010E0101205F5F
:10306000000E215BB8D7800E4B6E800E0101211936
:103070004B5C02E120510C0816E320C132F0F0EC69
:1030800007F029C14FF02AC150F02BC151F02CC1DB
:1030900052F068EC02F04BC029F14CC02AF14DC04F
:1030A0002BF14EC02CF129C14BF02AC14CF02BC1A1
:1030B0004DF02CC14EF04F6A506A516A526AAAEC28
:1030C00009F0000ED8A4010E4B6E4B52D8B478D044
:1030D00029C14BF02AC14CF02BC14DF02CC14EF050
:1030E000D1EC0AF0000E0101336F4E1808E13351A4
:1030F0004D1805E133514C1802E14B50000A60E1D4
:10310000800E4B6E800E2E194B5C02E12D51010892
:1031100057E22DC132F007EC05F04BC04FF04CC028
:1031200050F04DC051F04EC052F029C14BF02AC1B1
:103130004CF02BC14DF02CC14EF027EC0AF05F0E85
:103140004F6E700E506E090E516E810E526E93ECE2
:1031500004F0010ED8B0000E4B6E4B5206E0090E83
:1031600001012D5F000E2E5B05D00101080E2D5FC1
:10317000000E2E5B2DC132F007EC05F04BC04FF076
:103180004CC050F04DC051F04EC052F029C14BF030
:103190002AC14CF02BC14DF02CC14EF027EC0AF0A7
:1031A000D1EC0AF04BC02FF14CC030F14DC031F1E1
:1031B0004EC032F10101296B2A6B2B6B2C6B39D07D
:1031C00029C14BF02AC14CF02BC14DF02CC14EF05F
:1031D000D1EC0AF04BC02FF14CC030F14DC031F1B1
:1031E0004EC032F12FC14BF030C14CF031C14DF027
:1031F00032C14EF06EEC0BF04BC04FF04CC050F0B3
:103200004DC051F04EC052F029C14BF02AC14CF0D4
:103210002BC14DF02CC14EF082EC0BF04BC029F1CC
:103220004CC02AF14DC02BF14EC02CF101012D6B89
:103230002E6B010E226F22510A0A37E0020E4F6EEA
:1032400022C14BF0000E4C6E4D6E4E6E4F5007E09B
:103250004B364B904C364D364E36FF0FF8D7F20EAC
:103260004B264B0E4C22000E4D224BC0F6FF4CC09D
:10327000F7FF4DC0F8FF0900F5CF33F10900F5CF96
:1032800034F10900F5CF35F10900F5CF36F13651AB
:10329000325D08E13551315D05E13451305D02E1C7
:1032A00033512F5D02E3222BC6D7225120254B6ECE
:1032B000000E21214C6E2D514B262E514C224B508D
:1032C000235F4C50245B26B703D02051211104E02A
:1032D000010E235F000E245B030E25154B6E26C1E5
:1032E0004CF0000E4C164B504C1004E0010E235FC6
:1032F000000E245B25A549D025A31AD0010E251563
:103300004B6E26C14CF0000E4C164B504C1003E097
:103310002D0E4B6E02D02B0E4B6E2AC0E1FF2BC040
:10332000E2FF4BC0E6FF2A4A2B2A274B282B14D05A
:10333000010E25154B6E26C14CF0000E4C164B505D
:103340004C100AE02AC0E1FF2BC0E2FF200EE66E1F
:103350002A4A2B2A274B282B800E4B6E800E2419CD
:103360004B5C02E1235100080FE22AC0E1FF2BC0B1
:10337000E2FF300EE66E2A4A2B2A274B282B010E3D
:10338000235F000E245BE8D74AD025B718D0800E03
:103390004B6E800E24194B5C02E1235100080FE2B2
:1033A0002AC0E1FF2BC0E2FF200EE66E2A4A2B2A3C
:1033B000274B282B010E235F000E245BE8D725A3A3
:1033C0001AD0010E25154B6E26C14CF0000E4C167E
:1033D0004B504C1003E02D0E4B6E02D02B0E4B6E5B
:1033E0002AC0E1FF2BC0E2FF4BC0E6FF2A4A2B2A8E
:1033F000274B282B14D0010E25154B6E26C14CF0FF
:10340000000E4C164B504C100AE02AC0E1FF2BC0B6
:10341000E2FF200EE66E2A4A2B2A274B282B22C1D8
:103420004BF022074B5251E0020E4F6E22C14BF07F
:10343000000E4C6E4D6E4E6E4F5007E04B364B906B
:103440004C364D364E36FF0FF8D7F20E4B264B0E4C
:103450004C22000E4D224BC0F6FF4CC0F7FF4DC072
:10346000F8FF0900F5CF4FF00900F5CF50F0090043
:10347000F5CF51F00900F5CF52F02FC14BF030C11C
:103480004CF031C14DF032C14EF087EC0BF00A0E1A
:103490004F6E000E506E516E526E87EC0BF053C0A3
:1034A0004BF054C04CF055C04DF056C04EF0300EAD
:1034B0004B262AC0E1FF2BC0E2FF4BC0E6FF2A4AA1
:1034C0002B2A0101274B282BAAD7800E4B6E800E8A
:1034D0002E194B5C02E12D5100080FE22AC0E1FFDA
:1034E0002BC0E2FF300EE66E2A4A2B2A274B282BF0
:1034F000010E2D5F000E2E5BE8D7800E000A4B6E8A
:10350000800E21194B5C02E12051080803E2080EED
:10351000226F02D020C122F12251205F000E215BD8
:10352000225302E126A70AD02AC0E1FF2BC0E2FF06
:103530002E0EE66E2A4A2B2A274B282B22C132F068
:1035400007EC05F029C14FF02AC150F02BC151F012
:103550002CC152F07DEC01F011EC0DF04BC02FF1BD
:103560004CC030F14DC031F14EC032F10101225357
:1035700052E02207020E4F6E22C14BF0000E4C6E3D
:103580004D6E4E6E4F5007E04B364B904C364D36DD
:103590004E36FF0FF8D7F20E4B264B0E4C22000E84
:1035A0004D224BC0F6FF4CC0F7FF4DC0F8FF09009D
:1035B000F5CF4FF00900F5CF50F00900F5CF51F0ED
:1035C0000900F5CF52F02FC14BF030C14CF031C1A2
:1035D0004DF032C14EF087EC0BF00A0E4F6E000E2C
:1035E000506E516E526E87EC0BF053C04BF054C0CE
:1035F0004CF055C04DF056C04EF0300E4B262AC050
:10360000E1FF2BC0E2FF4BC0E6FF2A4A2B2A010153
:10361000274B282BABD7205121110FE02AC0E1FF07
:103620002BC0E2FF300EE66E2A4A2B2A274B282BAE
:10363000010E205F000E215BEED725A71AD0800E69
:103640004B6E800E24194B5C02E12351000811E2FD
:103650002AC0E1FF2BC0E2FF200EE66E2A4A2B2A89
:10366000274B282B010E235F000E245B23512411CE
:10367000EFE1CEEF0EF0C00E2515336F26C134F109
:10368000000E3417000E341902E1000E3319D8A4CD
:1036900081D025A929D02FC0E9FF30C0EAFFEECFA5
:1036A0004BF0EECF4CF04BC0E9FF4CC0EAFFEECF41
:1036B0002FF1EECF30F1EECF31F1EECF32F12FC05E
:1036C000E9FF30C0EAFFEECF4BF0EECF4CF0040E36
:1036D0004B26000E4C222FC0E1FF30C0E2FF4BC052
:1036E000E6FF4CC0E6FF2ED02FC0E9FF30C0EAFF56
:1036F000EECF4BF0EECF4CF04BC0E9FF4CC0EAFFF1
:10370000EECF2FF1EECF30F1000E30BFFF0E316F54
:10371000326F000E30BFFF0E316F326F2FC0E9FFE6
:1037200030C0EAFFEECF4BF0EECF4CF0020E4B264E
:10373000000E4C222FC0E1FF30C0E2FF4BC0E6FF7D
:103740004CC0E6FF800E32194B6E800E4B5C08E1D8
:10375000000E315D05E1000E305D02E1000E2F5DCF
:1037600018E2030E2513000E26134B6A4C6A4D6AAD
:103770004E6A2F514B5E30514C5A31514D5A325195
:103780004E5A4BC02FF14CC030F14DC031F14EC0FC
:1037900032F155D025A929D02FC0E9FF30C0EAFF6A
:1037A000EECF4BF0EECF4CF04BC0E9FF4CC0EAFF40
:1037B000EECF2FF1EECF30F1EECF31F1EECF32F18F
:1037C0002FC0E9FF30C0EAFFEECF4BF0EECF4CF058
:1037D000040E4B26000E4C222FC0E1FF30C0E2FF4A
:1037E0004BC0E6FF4CC0E6FF2AD02FC0E9FF30C037
:1037F000EAFFEECF4BF0EECF4CF04BC0E9FF4CC0F0
:10380000EAFFEECF2FF1EECF30F1000E316F326FC5
:10381000000E316F326F2FC0E9FF30C0EAFFEECFEC
:103820004BF0EECF4CF0020E4B26000E4C222FC078
:10383000E1FF30C0E2FF4BC0E6FF4CC0E6FF000EE8
:10384000211902E1000E20190FE1000E4B6E321912
:1038500008E14B50311905E14B50301902E12F516D
:10386000000A02E1204B212BC00E25154B6E4BC0E8
:1038700037F1B7D0010E226F22510A0A37E0020E4B
:103880004F6E22C14BF0000E4C6E4D6E4E6E4F507F
:1038900007E04B364B904C364D364E36FF0FF8D77F
:1038A000F20E4B264B0E4C22000E4D224BC0F6FF63
:1038B0004CC0F7FF4DC0F8FF0900F5CF33F1090008
:1038C000F5CF34F10900F5CF35F10900F5CF36F128
:1038D0003651325D08E13551315D05E13451305DDD
:1038E00002E133512F5D02E3222BC6D789D0010EAE
:1038F000226F2251080A37E0020E4F6E22C14BF0B0
:10390000000E4C6E4D6E4E6E4F5007E04B364B9096
:103910004C364D364E36FF0FF8D71A0E4B264C0E4E
:103920004C22000E4D224BC0F6FF4CC0F7FF4DC09D
:10393000F8FF0900F5CF33F10900F5CF34F10900A4
:10394000F5CF35F10900F5CF36F13651325D08E19A
:103950003551315D05E13451305D02E133512F5D68
:1039600002E3222BC6D74CD0010E226F22510C0A43
:1039700037E0020E4F6E22C14BF0000E4C6E4D6EC2
:103980004E6E4F5007E04B364B904C364D364E3610
:10399000FF0FF8D73A0E4B264C0E4C22000E4D224C
:1039A0004BC0F6FF4CC0F7FF4DC0F8FF0900F5CF44
:1039B00033F10900F5CF34F10900F5CF35F10900F5
:1039C000F5CF36F13651325D08E13551315D05E113
:1039D0003451305D02E133512F5D02E3222BC6D713
:1039E0000FD03751000AD8B445D73751C00AD8B4E0
:1039F00041D73751800AD8B47AD73751400AB4E05A
:103A0000800E4B6E800E21194B5C02E12051225D2D
:103A100003E220C122F10DD0800E21194B6E800EE1
:103A20004B5C02E12251205D04E222C120F1000E34
:103A3000216F235124110EE0030E25154B6E26C174
:103A40004CF0000E4C164B504C1004E0010E235F5E
:103A5000000E245B800E21194B6E800E24194B5CE6
:103A600002E12351205D05E22051235F2151245BB7
:103A700002D0236B246BC40E2515336F2651080B1F
:103A8000346F3451080A02E1400E331908E1235122
:103A9000241104E0010E235F000E245B1CD0C00E35
:103AA0002515336F2651080B346F3451080A02E193
:103AB000800E331910E1800E4B6E800E24194B5C82
:103AC00002E12351020805E2020E235F000E245B8F
:103AD00002D0236B246B25A56DD025A31AD0010E2F
:103AE00025154B6E26C14CF0000E4C164B504C1059
:103AF00003E02D0E4B6E02D02B0E4B6E2AC0E1FF61
:103B00002BC0E2FF4BC0E6FF2A4A2B2A274B282B6B
:103B10003CD0010E25154B6E26C14CF0000E4C1604
:103B20004B504C100BE02AC0E1FF2BC0E2FF200EEF
:103B3000E66E2A4A2B2A274B282B27D0C00E2515A4
:103B4000336F2651080B346F3451080A02E1800E9E
:103B500033191BE12AC0E1FF2BC0E2FF300EE66EF5
:103B60002A4A2B2A274B282B25AB03D0580E4B6E05
:103B700002D0780E4B6E2AC0E1FF2BC0E2FF4BC093
:103B8000E6FF2A4A2B2A274B282B2351241111E028
:103B90002AC0E1FF2BC0E2FF300EE66E2A4A2B2A34
:103BA000274B282B010E235F000E245B2351241189
:103BB000EFE184D02351241113E025B711D02AC09E
:103BC000E1FF2BC0E2FF200EE66E2A4A2B2A274B8C
:103BD000282B010E235F000E245B23512411EFE1FB
:103BE00025A31AD0010E25154B6E26C14CF0000EF0
:103BF0004C164B504C1003E02D0E4B6E02D02B0E8A
:103C00004B6E2AC0E1FF2BC0E2FF4BC0E6FF2A4A01
:103C10002B2A274B282B14D0010E25154B6E26C1BD
:103C20004CF0000E4C164B504C100AE02AC0E1FF3D
:103C30002BC0E2FF200EE66E2A4A2B2A274B282BA8
:103C4000C00E2515336F2651080B346F3451080A06
:103C500002E1400E33190BE12AC0E1FF2BC0E2FF65
:103C6000300EE66E2A4A2B2A274B282B27D0C00E6F
:103C70002515336F2651080B346F3451080A02E1C1
:103C8000800E33191BE12AC0E1FF2BC0E2FF300E8A
:103C9000E66E2A4A2B2A274B282B25AB03D0580E39
:103CA0004B6E02D0780E4B6E2AC0E1FF2BC0E2FFB4
:103CB0004BC0E6FF2A4A2B2A274B282B800E4B6E3F
:103CC000800E21194B5C02E12051225D0BE22AC0DB
:103CD000E1FF2BC0E2FF300EE66E2A4A2B2A274B6B
:103CE000282BECD720C14BF021C14CF0010E205FF6
:103CF000000E215B4B504C10D8B446D1C00E251598
:103D00004B6E4BC033F124D1020E4F6E20C14BF0ED
:103D100021C14CF0000E21BFFF0E4D6E4E6E4F5074
:103D200007E04B364B904C364D364E36FF0FF8D7EA
:103D3000F20E4B264B0E4C22000E4D224BC0F6FFCE
:103D40004CC0F7FF4DC0F8FF0900F5CF4FF0090058
:103D5000F5CF50F00900F5CF51F00900F5CF52F042
:103D60002FC14BF030C14CF031C14DF032C14EF09B
:103D700087EC0BF00A0E4F6E000E506E516E526EB5
:103D800087EC0BF053C04BF054C04CF055C04DF0D5
:103D900056C04EF0300E4B240101226FE9D025AB06
:103DA0004CD0020E4F6E20C14BF021C14CF0000EE2
:103DB00021BFFF0E4D6E4E6E4F5007E04B364B90BD
:103DC0004C364D364E36FF0FF8D71A0E4B264C0E9A
:103DD0004C22000E4D224BC0F6FF4CC0F7FF4DC0E9
:103DE000F8FF0900F5CF4FF00900F5CF50F00900BA
:103DF000F5CF51F00900F5CF52F02FC14BF030C193
:103E00004CF031C14DF032C14EF087EC0BF00F0E8B
:103E10004B16000E4C164D164E166A0E4B264C0EC7
:103E20004C22000E4D224BC0F6FF4CC0F7FF4DC098
:103E3000F8FF0900F5CF22F14CD0020E4F6E20C1E1
:103E40004BF021C14CF0000E010121BFFF0E4D6E61
:103E50004E6E4F5007E04B364B904C364D364E363B
:103E6000FF0FF8D71A0E4B264C0E4C22000E4D2297
:103E70004BC0F6FF4CC0F7FF4DC0F8FF0900F5CF6F
:103E80004FF00900F5CF50F00900F5CF51F00900CF
:103E9000F5CF52F02FC14BF030C14CF031C14DF095
:103EA00032C14EF087EC0BF00F0E4B16000E4C1685
:103EB0004D164E167C0E4B264C0E4C22000E4D22FB
:103EC0004BC0F6FF4CC0F7FF4DC0F8FF0900F5CF1F
:103ED00022F14ED0020E4F6E20C14BF021C14CF0AA
:103EE000000E010121BFFF0E4D6E4E6E4F5007E0D8
:103EF0004B364B904C364D364E36FF0FF8D73A0EB8
:103F00004B264C0E4C22000E4D224BC0F6FF4CC0EF
:103F1000F7FF4DC0F8FF0900F5CF4FF00900F5CFCE
:103F200050F00900F5CF51F00900F5CF52F02FC144
:103F30004BF030C14CF031C14DF032C14EF087EC46
:103F40000BF0070E4B140101226F300E222710D008
:103F500001013351000AD8B4D7D63351C00AD8B4BE
:103F6000D3D63351800AD8B41AD73351400AB2E0BD
:103F70002AC0E1FF2BC0E2FF22C1E6FF2A4A2B2A1A
:103F80000101274B282BAED6010125A71BD0800E9F
:103F90004B6E800E24194B5C02E12351000812E2A3
:103FA0002AC0E1FF2BC0E2FF200EE66E2A4A2B2A30
:103FB0000101274B282B010E235F000E245B2351A8
:103FC0002411EEE1CEEF0EF027C14BF028C14CF0EA
:103FD0001200006A2AC032F0ABEC0DF0010E006E48
:103FE00012001B6A1C6A030EC26EC2B2FED7C4CF97
:103FF0001BF0000E1C6E1BC04CF04B6A4BC01BF03C
:104000004CC01CF0C3504B12000E4C1212000001A9
:104010004B50536E4C504B6E4C6A4D6A4E6A566A0A
:10402000576A960E4E6E556A4BC04CF053C04BF01B
:10403000536A4D6AF0EC0DF012001BC04FF01CC02B
:1040400050F01DC051F01EC052F04B6A4C6A4D6AD0
:104050004E6A93EC04F0000ED8B0010E4B6E4B523A
:1040600005E04B6A4C6A4D6A4E6A12001BC01FF095
:104070001CC020F01DC021F01EC022F0000E4F6EAB
:10408000000E506E000E516E7F0E526E1BC04BF034
:104090001CC04CF01DC04DF01EC04EF093EC04F05F
:1040A000010ED8B0000E4B6E4B521AE01FC04FF0FD
:1040B00020C050F021C051F022C052F0000E4B6ED3
:1040C000000E4C6E000E4D6E7F0E4E6E27EC0AF009
:1040D0004BC01FF04CC020F04DC021F04EC022F06C
:1040E0001FC02AF020C02BF021C02CF022C02DF0E0
:1040F000280E2E6E000E2F6E2DEC0EF04BC01FF012
:104100004CC020F04DC021F04EC022F04BC02AF030
:104110004CC02BF04DC02CF04EC02DF0020E4F6E57
:10412000000E506E28C04BF029C04CF0C2EC09F0D4
:104130004BC02EF04CC02FF057EC0EF04BC01FF0D0
:104140004CC020F04DC021F04EC022F0000E4F6E4A
:10415000000E506E000E516E7F0E526E1BC04BF063
:104160001CC04CF01DC04DF01EC04EF093EC04F08E
:10417000010ED8B0000E4B6E4B521AE01FC04FF02C
:1041800020C050F021C051F022C052F0000E4B6E02
:10419000000E4C6E000E4D6E7F0E4E6E27EC0AF038
:1041A0004BC01FF04CC020F04DC021F04EC022F09B
:1041B000140E276E1FC04FF020C050F021C051F0E8
:1041C00022C052F01BC04BF01CC04CF01DC04DF083
:1041D0001EC04EF027EC0AF01FC04FF020C050F078
:1041E00021C051F022C052F068EC02F0000E4F6E78
:1041F000000E506E000E516E800E526E27EC0AF0CB
:104200004BC023F04CC024F04DC025F04EC026F02A
:104210001FC04FF020C050F021C051F022C052F01A
:10422000AAEC09F0010ED8A4000E4B6E4B520BE124
:1042300023C01FF024C020F025C021F026C022F0AA
:1042400027062752B7E11FC04BF020C04CF021C019
:104250004DF022C04EF01200200E266E000E276E8A
:104260001BC02AF01CC02BF01DC02CF01EC02DF06E
:104270001FC02EF0260E2F6E000E306EBCEC0EF01E
:104280004BC024F04CC025F04B501B24E16E4C5029
:104290001C20E26EE66A24C04BF025C04CF01200F0
:1042A0001D6A1E6A1D501B24E96E1E501C20EA6EFA
:1042B000EECF4BF04B520DE01D501B24E96E1E500B
:1042C0001C20EA6EEECF2AF0E9EC1FF01D4A1E2AF0
:1042D000E9D712000FD0800E1B6E19D0C00E1B6ED6
:1042E00016D0940E1B6E13D0D40E1B6E10D0800E01
:1042F0001B6E0DD01B50010AEEE01B50020AEEE0CF
:104300001B50030AEEE01B50040AEEE0F0D71C0439
:104310004B6E1B504B264BC01BF04BC032F0ABEC2E
:104320000DF0006A1F6A206A1F501D24E96E20509C
:104330001E20EA6EEECF4BF04B520DE01F501D24B5
:10434000E96E20501E20EA6EEECF32F0ABEC0DF09D
:104350001F4A202AE9D7010E006E120017C001F093
:1043600018C002F017C0E1FF18C0E2FFE66A17C0EC
:1043700001F018C002F0110EE126E76A120EE15EAC
:104380007EEC04F0E78AE788E7867CEC04F0E796A9
:104390007EEC04F0E78AE788E7867CEC04F0E79699
:1043A0008DEC04F08DEC04F0E78AE788E7867CEC7E
:1043B00004F0E7967EEC04F0E78AE798E7867CEC69
:1043C00004F0E7968DEC04F0E78AE798E7867CEC4A
:1043D00004F0E796E78EE79CE7867CEC04F0E7962E
:1043E0008DEC04F0000EE76EE7867CEC04F0E796B7
:1043F000E78EE78CE78AE788E7867CEC04F0E796AF
:104400008DEC04F0000EE76EE7867CEC04F0E79696
:10441000E788E7867CEC04F0E7967EEC04F0000E7B
:10442000E76EE7867CEC04F0E796E78CE78AE786A0
:104430007CEC04F0E7968DEC04F0010E006E1200A7
:10444000176A186AF1EC1FF0000E4F6E4C504F5C6B
:1044500002E14B5003080CE2800E18184B6E800EE0
:104460004B5C02E1400E175C03E2174A182AEAD7B8
:10447000176A186A800E18184B6E800E4B5C02E1AA
:10448000200E175C26E2020E4F6E17C04BF018C0CC
:104490004CF04F5005E04B364B904C36FF0FFAD79F
:1044A000600E4B24196E000E4C201A6EF1EC1FF0BA
:1044B00007EC20F019C0E1FF1AC0E2FF4BC0E6FF95
:1044C0004CC0E6FF4DC0E6FF4EC0E6FF174A182A73
:1044D000D1D712000101016B026B036B046B056BFA
:1044E000066B076B086B096B0A6B0B6B0C6B0D6B28
:1044F0000E6B0F6B106B0001E06B200E0001E05D96
:10450000D8B039D1020E4F6EE0C015F1000E010196
:10451000166F176F186F4F5008E00101153715918E
:10452000163717371837FF0FF7D78E0E01011525ED
:104530004B6E4C0E16214C6E000E17214D6E000E68
:104540004BC0F6FF4CC0F7FF4DC0F8FF0900F5CF98
:104550004FF00900F5CF50F00900F5CF51F00900F8
:10456000F5CF52F0600E1525E96E000E1621EA6EA9
:10457000EECF4BF0EECF4CF0EECF4DF0EECF4EF055
:104580007DEC01F0520E4F6EB80E506E1E0E516E45
:104590007D0E526E7DEC01F001C14FF002C150F072
:1045A00003C151F004C152F068EC02F04BC001F1BC
:1045B0004CC002F14DC003F14EC004F10E0E0101DA
:1045C00015254B6E4D0E16214C6E000E17214D6EAB
:1045D000000E4BC0F6FF4CC0F7FF4DC0F8FF0900BE
:1045E000F5CF4FF00900F5CF50F00900F5CF51F0AD
:1045F0000900F5CF52F0600E1525E96E000E162168
:10460000EA6EEECF4BF0EECF4CF0EECF4DF0EECFAA
:104610004EF07DEC01F0520E4F6EB80E506E1E0E35
:10462000516E7D0E526E7DEC01F005C14FF006C15A
:1046300050F007C151F008C152F068EC02F04BC0D5
:1046400005F14CC006F14DC007F14EC008F18E0EC9
:10465000010115254B6E4D0E16214C6E000E1721D3
:104660004D6E000E4BC0F6FF4CC0F7FF4DC0F8FF7B
:104670000900F5CF4FF00900F5CF50F00900F5CF54
:1046800051F00900F5CF52F0600E1525E96E000ECD
:104690001621EA6EEECF4BF0EECF4CF0EECF4DF0A0
:1046A000EECF4EF07DEC01F0520E4F6EB80E506E14
:1046B0001E0E516E7D0E526E7DEC01F009C14FF061
:1046C0000AC150F00BC151F00CC152F068EC02F07D
:1046D0004BC009F14CC00AF14DC00BF14EC00CF1BA
:1046E0000E0E010115254B6E4E0E16214C6E000E5E
:1046F00017214D6E000E4BC0F6FF4CC0F7FF4DC0AA
:10470000F8FF0900F5CF4FF00900F5CF50F0090090
:10471000F5CF51F00900F5CF52F0600E1525E96E86
:10472000000E1621EA6EEECF4BF0EECF4CF0EECF3E
:104730004DF0EECF4EF07DEC01F0520E4F6EB80E04
:10474000506E1E0E516E7D0E526E7DEC01F00DC14D
:104750004FF00EC150F00FC151F010C152F068EC93
:1047600002F04BC00DF14CC00EF14DC00FF14EC028
:1047700010F1E02BC2D601C14BF002C14CF003C1D5
:104780004DF004C14EF001C14FF002C150F003C121
:1047900051F004C152F07DEC01F04BC015F14CC05A
:1047A00016F14DC017F14EC018F105C14BF006C10E
:1047B0004CF007C14DF008C14EF005C14FF006C1E5
:1047C00050F007C151F008C152F07DEC01F015C165
:1047D0004FF016C150F017C151F018C152F068ECFB
:1047E00002F04BC01BF04CC01CF04DC01DF04EC081
:1047F0001EF01DEC20F04BC001F14CC002F14DC089
:1048000003F14EC004F1000E4F6E000E506E000E0C
:10481000516E7B0E526E7DEC01F04BC001F14CC02D
:1048200002F14DC003F14EC004F109C14BF00AC1C1
:104830004CF00BC14DF00CC14EF009C14FF00AC154
:1048400050F00BC151F00CC152F07DEC01F04BC0A7
:1048500015F14CC016F14DC017F14EC018F10DC145
:104860004BF00EC14CF00FC14DF010C14EF00DC118
:104870004FF00EC150F00FC151F010C152F07DEC5D
:1048800001F015C14FF016C150F017C151F018C119
:1048900052F068EC02F04BC01BF04CC01CF04DC055
:1048A0001DF04EC01EF01DEC20F04BC009F14CC0B5
:1048B0000AF14DC00BF14EC00CF1000E4F6E000E10
:1048C000506E000E516E7B0E526E7DEC01F04BC0AF
:1048D00009F14CC00AF14DC00BF14EC00CF1000EB5
:1048E0004F6E000E506E480E516E850E526E7DEC6E
:1048F00001F001C14FF002C150F003C151F004C1F9
:1049000052F027EC0AF04BC011F14CC012F14DC02F
:1049100013F14EC014F14BC04FF04CC050F04DC0DD
:1049200051F04EC052F0000E4B6E000E4C6E200E39
:104930004D6E820E4E6E93EC04F0010ED8B0000E58
:104940004B6E4B5218E1000E4F6E000E506E200E53
:10495000516E830E526E01C14BF002C14CF003C187
:104960004DF004C14EF093EC04F0010ED8B0000EEF
:104970004B6E4B521AE0829E4F6A82BE4F2A000E47
:104980004FB0400E8218400B821A820E566EFF0EF8
:10499000556E562E01D003D0552EFED7FAD7870E6E
:1049A000556E552EFED700000AD0828E4F6A82BE09
:1049B0004F2A000E4FB0400E8218400B821AE10EB3
:1049C0001B6E000E1C6E8E0E1D6E4E0E1E6E000EA9
:1049D0001F6E01C120F002C121F003C122F004C109
:1049E00023F02CEC21F0800E326EABEC0DF0E10EDA
:1049F0001B6E000E1C6E50EC21F0E10E1B6E000EC3
:104A00001C6E980E1D6E4E0E1E6E000E1F6E09C19E
:104A100020F00AC121F00BC122F00CC123F02CECD4
:104A200021F0C00E326EABEC0DF0E10E1B6E000EED
:104A30001C6E50EC21F0E10E1B6E000E1C6EA20EDF
:104A40001D6E4E0E1E6E000E1F6E11C120F012C1A3
:104A500021F013C122F014C123F02CEC21F0020E3E
:104A60001B6E0A0E1C6EE10E1D6E000E1E6E6AECB1
:104A700021F01200480E036E610E046E720E056E78
:104A80006D0E066E6F0E076E6E0E086E690E096E65
:104A9000630E0A6E200E0B6E440E0C6E650E0D6ECC
:104AA000740E0E6E650E0F6E630E106E740E116E28
:104AB0006F0E126E720E136E146A030E156E000ED8
:104AC000166E12003AEC25F0820E566EFF0E556EF1
:104AD000562E01D003D0552EFED7FAD7870E556E2D
:104AE000552EFED700000E0EC16EC26A920EC06E29
:104AF000FF0E926E936AFF0E826E020E946E829E7D
:104B00004C6A82BE4C2A000E4CB0400E8218400BFC
:104B1000821A060E576EFF0E566EFF0E556E572EFA
:104B200001D007D0562E01D003D0552EFED7FAD78C
:104B3000F6D71A0E566EFF0E556E562E01D003D0C4
:104B4000552EFED7FAD7420E556E552EFED7828EC1
:104B50004C6A82BE4C2A000E4CB0400E8218400BAC
:104B6000821A810E176E0F0E186EAEEC21F0010E38
:104B7000326EABEC0DF00C0E326EABEC0DF020ECA7
:104B800022F06AEC22F0FBD7FFD70000007FCDCCEB
:104B90004C7B0AD723786F12037517B75171ACC5D8
:104BA000276EBD37066B95BF566777CC2B645F7059
:104BB0000961FFE65B5D08E53C3C6042221B0000AA
:104BC000007F000020820000488500007A880040B5
:104BD0001C8C0050438F002474928096189620BC41
:104BE0003E99286B6E9CF90215A0EC782DC1CAF293
:104BF00049E2010000000A00000064000000E80330
:104C0000000010270000A086010040420F0080969F
:104C1000980000E1F50500CA9A3B01000000100071
:104C20000000000100000010000000000100000072
:104C3000100000000001000000100100000008004A
:104C40000000400000000002000000100000008092
:104C5000000000000400000020000000000100002F
:104C600000080000004000000000303132333435CD
:104C70003637383941424344454600FF30313233FC
:104C800034353637383961626364656600FF000089
:104C90000000CFBC487B5CC5477CE79F147DB6EE27
:104CA000437D785A717D99390E7E5367227EAA041E
:104CB000357EBAE3457EE9DA547E55C5617E2383AD
:104CC0006C7EDAF9747E9B147B7E5AC47E7E000073
:104CD000007F83C47E7EEC147B7E52FA747EC18397
:104CE0006C7E18C6617ECFDB547EC0E4457ECF0566
:104CF000357E9368227EF13A0E7E515D717DB2F170
:104D0000437DFFA2147DB3CB477CACC9487B000038
:104D1000007F6EC47E7EC4147B7E16FA747E72831E
:104D20006C7EB6C5617E5CDB547E3DE4457E3C0511
:104D3000357EF367227E453A0E7EE55B717D34F069
:104D4000437D73A1147D88C8477C3DC3487B34CF25
:104D50004E6E60B6C87B31C2C77C5B9E947D38EDD9
:104D6000C37D0B59F17DED388E7EB366A27E1804AB
:104D7000B57E36E3C57E77DAD47EF3C4E17ED48295
:104D8000EC7E9EF9F47E7314FB7E46C4FE7E00002A
:104D90000000E79F147D99390E7EBAE3457E238398
:104DA0006C7E5AC47E7EEC147B7E18C6617ECF0575
:104DB000357E515D717DB3CB477CF2AFC87BB9EBDB
:104DC000C37D1366A27E04DAD47E62F9F47E00000D
:104DD000807FCAFAF47EB5DCD47ED369A27EAEF4BD
:104DE000C37D89D6C87BAFB8477CC554717D61024D
:104DF000357ECFC3617EFA137B7ED4C47E7EFE8473
:104E00006C7ECDE6457EA13D0E7E2EA9147D000070
:104E1000007F16FA747E5CDB547EF367227E34F0EA
:104E2000437D3DC3487B31C2C77C0B59F17D1804DB
:104E3000B57EF3C4E17E7314FB7E97C4FE7E1184BD
:104E4000EC7E43E5C57E9D3B8E7E8BA4947D671BE7
:104E50009B70449B147D95370E7E30E2457E3682F2
:104E60006C7E1DC47E7E65157B7E3CC7617E85079A
:104E7000357E9861717D35D5477CA69CC87B3FE720
:104E8000C37D3464A27EABD8D47EAEF8F47E317399
:104E9000743D252E316600FF3372643D252E316648
:104EA00000FF5448443D252E316600FF00000000FD
:104EB000A3147383FEE87184A2F9338510436D85D2
:104EC000C7211286C0392C861FA94486A6335B866B
:104ED000C3A16F868BE000877AB2088766330F879D
:104EE000475314877A051887E3401A8700001B8709
:104EF000FB401A87AB05188790531487C6330F877A
:104F0000F0B2088716E1008700A36F8608355B863C
:104F1000A2AA4486603B2C8680231286AD466D850E
:104F200061FD3385ABF071843624738300002082E9
:104F300000002082000020820000208200002082E9
:104F400000002082000020820000208200002082D9
:104F500000002082000020820000208200002082C9
:104F600000002082000020820000208200002082B9
:104F700000002082000020820000208200002082A9
:104F800000002082000020820000208200001082A9
:104F90000000008200000082000000820000008209
:104FA000000060810000608100006081FFFFFFFF62
:020000040030CA
:0E000000FFF8FFFEFFFFBBFFFFFFFFFFFFFF4C
:00000001FF
